:020000040000FA
:040000008A115228E7
:08000800FE00030E8301A300BA
:100010000A08A4008A014D28820700340034003405
:100020000034003400340034003400340034003430
:10003000003400340034013400340034003400341F
:1000400002340034033404340034003405340634FC
:1000500000340734003400340034003400340034F9
:100060000834003409340A34003400340B340C34BE
:1000700000340D34003400340034003400340E34C5
:1000800000340F34003400340034003400340034C1
:10009000003400340034003400340408A600200882
:1000A000A200192A83169F0183129F019A019C01C5
:1000B0008316051405118510363095008113D0285C
:1000C0000130900050308E00FB308F004C14CC106B
:1000D0007D117D0885004C11B001B10183160C1013
:1000E0000B178B170800831227100C1C7C28831613
:1000F0000C1C7C28831227148312271CB5280C1093
:100100004C1C952850308E00FB308F003008310495
:10011000031D90286230B0000330B1004C10A428B9
:10012000B003300A0319B103A428F8308E008F0001
:1001300030083104031DA028CC1083160C10A4280D
:10014000B003300A0319B1038312CC1CAD284C1D37
:10015000AB284C11AE284C15AE284C114C19B228C6
:100160007D11B3287D157D0885002208A000260892
:10017000840024088A00230E8300FE0E7E0E0900F0
:10018000CC18CF284C141430B0000530B1005030DA
:100190008E00FB308F00CC140C1083160C1408005A
:1001A0008312CC124C13C201C301CC134D10CD10DD
:1001B000C401C501C601CA01CB01232ADA005808CF
:1001C000DD00DA065A0EF039DD00DA065A08DB00E7
:1001D000DC015B08DE00DD015908DF00E0015F089B
:1001E0005D04E10060085E04E20003105C0CE400C2
:1001F0005B0CE3000330A0000310E40CE30CA00B45
:10020000FC2863086106E50064086206E600031046
:100210005B0DE7005C0DE8000310E70DE80D03102F
:10022000E70DE80D67086506E90068086606EA005C
:100230006908A0006A08A1000800CC1AC30A0315C7
:10024000CC1E25294C1F262927294C1B03110319D5
:1002500038295030420203193229031832290B3051
:10026000C20734291D30C2074C13CC1A4C173A2947
:100270001430C207A030420203194029031CAF29E1
:100280000310C50CC40C0530430203194929031C93
:100290004A29C515A030C202C301CC1FA329C60A32
:1002A0000C30460203195629031CAF293F30440580
:1002B000A900AA0100308A0029080C208312A0009E
:1002C000200EF039AB000310450CAD00440CAC001F
:1002D0000530A0000310AD0CAC0CA00B6A29003057
:1002E0008A002C080C208312A0002B04A8004B08C5
:1002F000031D92292808CA0004304A022E1303194C
:100300008329031C2E1706304A02AE1303198A29CB
:100310000318AE172F102E1FAE1B2F142F1C92295F
:10032000CC13080036304B07840083132808800064
:10033000CB0A4B084A0203199F290318A129CC13A1
:100340004D14C601080038304402A0000B304502AD
:100350002004031DAF29CC17C601CB014D100800A6
:10036000D000FC3092058730920550088316920029
:100370008312121583168C140B178B170800831227
:10038000CF00B0298312CD18C729CD14CC13080093
:10039000CF00FF30D000D1004D18D0292010172AEF
:1003A00003304B02D2004F0852020319DB29031815
:1003B000DB295208CF004F08D500D301EE29530A9C
:1003C000D40036305407840083130008A00047305F
:1003D00053078400831320088000D30A5308550272
:1003E000031DDF294B08D600D301062A5008D80088
:1003F0005108D90036305307840083130008DE20EB
:1004000083122008D0002108D100D30A53085602D5
:10041000031DF6294D10B8305002A000F0305102F3
:1004200020045712031957162010571A20144F088A
:1004300008008C1C73288C10CD1C7328CC12051856
:10044000CC161D2173286020FA30BF21C2218312EF
:10045000CC114C12FD107D088500B301B401B5012B
:10046000831203139330A0001A30A1000A128A11DC
:10047000A10B362A0A128A11A00B342A00000000B0
:100480000000000000000330B200C8218312B20057
:100490004D1120184D154D1D702A03303202CD111B
:1004A0000319CD1547034D1203194D16CD16CD195D
:1004B0004D1ECD1248034D1303194D17CD17CD1AFC
:1004C0004D1FCD13490835024E10031D4E14CE1496
:1004D000CD1B4E1CCE10CE1C702A4908B500CC1581
:1004E000CC1D782ACC11C0208312B3010A30B4008D
:1004F0003308031D892A3408031D802A4C128A2AD6
:100500004C1E842A4C12852A4C16B4033230B30098
:100510008A2AB3034C1A8E2AFD108F2AFD147D08F7
:040520008500302AF8
:02400E00C43FAD
:00000001FF
